:100000000C9485070C94AD070C94AD070C94AD07C8
:100010000C94AD070C94AD070C94AD070C94AD0790
:100020000C94AD070C94AD070C9408120C94771245
:100030000C94AD070C94AD070C94AD070C94AD0770
:100040000C94AD070C94AD070C94AD070C94AD0760
:100050000C94AD070C94AD070C94AD070C94A91447
:100060000C94AD070C94AD070C94AD070C94AD0740
:100070000C94AD070C94AD070C94AD070C94AD0730
:100080000C94F3140C94AD070C94AD070C94AD07CD
:100090000C94AD070C94AD070C94AD070C94AD0710
:1000A0000C94AD070C94AD070C94AD0705A84CCD8E
:1000B000B2D44EB93836A9020C50B9918688083CA2
:1000C000A6AAAA2ABE000000803F423A0021424F61
:1000D00053532100483A0000000000003E5B4F5B94
:1000E0003E3E6B4F6B3E1C3E7C3E1C183C7E3C18DB
:1000F0001C577D571C1C5E7F5E1C00183C1800FFBF
:10010000E7C3E7FF0018241800FFE7DBE7FF3048EC
:100110003A060E2629792926407F050507407F05E6
:10012000253F5A3CE73C5A7F3E1C1C08081C1C3EDD
:100130007F14227F22145F5F005F5F06097F017FCB
:10014000006689956A606060606094A2FFA294086E
:10015000047E040810207E201008082A1C08081CB1
:100160002A08081E101010100C1E0C1E0C30383EF1
:100170003830060E3E0E06000000000000005F0052
:10018000000007000700147F147F14242A7F2A121E
:100190002313086462364956205000080703000004
:1001A0001C2241000041221C002A1C7F1C2A080836
:1001B0003E08080080703000080808080800006049
:1001C000600020100804023E5149453E00427F4035
:1001D0000072494949462141494D331814127F1094
:1001E00027454545393C4A494931412111090736DE
:1001F00049494936464949291E000014000000407B
:100200003400000008142241141414141400412274
:10021000140802015909063E415D594E7C12111223
:100220007C7F494949363E414141227F4141413E1F
:100230007F494949417F090909013E414151737F85
:100240000808087F00417F41002040413F017F08AE
:100250001422417F404040407F021C027F7F0408FF
:10026000107F3E4141413E7F090909063E4151212F
:100270005E7F09192946264949493203017F010356
:100280003F4040403F1F2040201F3F4038403F63D9
:100290001408146303047804036159494D43007F33
:1002A0004141410204081020004141417F04020104
:1002B00002044040404040000307080020545478A6
:1002C000407F284444383844444428384444287FF4
:1002D000385454541800087E090218A4A49C787F4E
:1002E0000804047800447D40002040403D007F1019
:1002F00028440000417F40007C047804787C080496
:1003000004783844444438FC182424181824241849
:10031000FC7C08040408485454542404043F442436
:100320003C4040207C1C2040201C3C4030403C4451
:10033000281028444C9090907C4464544C4400080D
:10034000364100000077000000413608000201023B
:1003500004023C2623263C1EA1A161123A40402003
:100360007A3854545559215555794121545478417E
:10037000215554784020545579400C1E5272123940
:1003800055555559395454545939555454580000F9
:10039000457C410002457D420001457C40F0292416
:1003A00029F0F0282528F07C545545002054547C31
:1003B000547C0A097F493249494932324848483217
:1003C000324A4848303A4141217A3A424020780046
:1003D0009DA0A07D39444444393D4040403D3C24EB
:1003E000FF2424487E4943662B2FFC2F2BFF09292D
:1003F000F620C0887E090320545479410000447DD2
:10040000413048484A32384040227A007A0A0A721B
:100410007D0D19317D2629292F28262929292630C5
:10042000484D4020380808080808080808382F10E8
:10043000C8ACBA2F102834FA00007B000008142A38
:10044000142222142A14089500220095AA005500AF
:10045000AAAA55AA55AA000000FF00101010FF001C
:10046000141414FF001010FF00FF1010F010F0140F
:100470001414FC001414F700FF0000FF00FF141414
:10048000F404FC141417101F10101F101F14141460
:100490001F00101010F0000000001F101010101F9F
:1004A00010101010F010000000FF101010101010AD
:1004B000101010FF10000000FF140000FF00FF00EC
:1004C000001F10170000FC04F41414171017141464
:1004D000F404F40000FF00F714141414141414F7B7
:1004E00000F7141414171410101F101F141414F410
:1004F000141010F010F000001F101F0000001F1457
:10050000000000FC140000F010F01010FF10FF14A9
:100510001414FF141010101F00000000F010FFFF53
:10052000FFFFFFF0F0F0F0F0FFFFFF000000000021
:10053000FFFF0F0F0F0F0F38444438447C2A2A3E28
:10054000147E02020606027E027E02635549416362
:100550003844443C04407E201E2006027E0202995C
:10056000A5E7A5991C2A492A1C4C7201724C304AF5
:100570004D4D303048784830BC625A463D3E49497E
:1005800049007E0101017E2A2A2A2A2A44445F4426
:100590004440514A444040444A51400000FF010356
:1005A000E080FF000008086B6B0836123624360620
:1005B0000F090F060000181800000010100030404E
:1005C000FF0101001F01011E00191D1712003C3C14
:1005D0003C3C0000000000F0F89C8E8783878E9CD6
:1005E000F8F00000FEFF0303030303070EFCF8000E
:1005F00000FEFF0303030303070EFCF80000FFFFE8
:1006000000000000000000FFFF0000FEFF83838366
:100610008383C7EE7C380000F8FC0E070303030752
:100620000EFCF800003F7FE0C08080C0E07F3FFF0D
:10063000FF01010101010101FFFF0000FFFF0C0CA0
:100640000C0C1C3E77E3C100007FFFC0C0C0C0C0DF
:10065000E0703F1F00001F3F70E0C0C0C0E0703F6F
:100660001F00007FFFC1C1C1C1C1E3773E1C000074
:100670001F3F70E0C0C0C0E0703F1F0000000000DE
:1006800001FFFF01000000D5F08D14A1C881CFD972
:10069000F1AF20002C0114006400140000000000E1
:1006A00064001400500014003C0014009600320056
:1006B0002800640000000000640032000000000018
:1006C000C80064009600640000000000E8031E00FB
:1006D000000000005052455353204120544F2052F7
:1006E0004553544152540053434F52453A2000471A
:1006F000414D45204F5645520020204D454E550056
:100700003E204D454E55002020524553554D450045
:100710003E20524553554D4500533A00483A004358
:10072000484F4F53452053484950000601C8004ADE
:1007300001C8008801C800EE0190018801C8004A84
:1007400001C800060190010000C800DC00C80006D6
:1007500001C8004A01C800B801900100805052450C
:100760005353204120544F205354415254004F467C
:1007700046004F4E00534E443A0048493A00703507
:1007800000000080C0E0F0F0F0F0F0F0F0F0F0F0E9
:10079000F0F0F0F0F07038081CFFDCE8F8F0F0F052
:1007A000F0F0F0F0F0F0F0F0F0F0E0C080000000C9
:1007B00000000000000080C0E0F0F0F0F0F0F0F089
:1007C000F0F0F0E000000080C0E0F0F0F0F0F0F0B9
:1007D000F0F0F0F0F0F0F0F070301000E0F0F0F039
:1007E000F0F0F0F0F0F0F0F0F0F0F0F0F070301029
:1007F00000001F3F7FFFFFFFF9F1F1F1F1F1F1F18F
:10080000F1F1F1F1E0C0800000FCFDFDFDFDFDE136
:10081000E1E1E1E1E1E1E1F1FFFFFFFF7F3F000006
:10082000E0F0F8FCFEFF7F3F9FCFE7E3E1E0E0FF71
:10083000FFFFFFFF0000FFFFFFFFFFFF01010101BE
:10084000010101010101010000000000FFFFEFE7CD
:10085000D738D1E1E1F1F1F171311101000000006F
:100860000080C0E0F0F0F1F1F1F1F1F1F1F1F1F11E
:10087000F9FFFFFF7F3F1F0000FFFFFFFF7F7F03A8
:100880000303030303030303030301000000000049
:100890007FFFFFFFFF00020303030303030303FFC4
:1008A000FFFFFF7F00001F3F7FFFFFFFF8F0F0F02A
:1008B000F0F0F0F0F0F0F07030100000FFFFFFFFFC
:1008C000FFFFF1F1F1F1F1F0F0F0F0F0F070301025
:1008D0000101010101010101010101010101010108
:1008E0000101010000008080E0E7F301000000004A
:1008F0008080E0E0F0000000000080E0E0F0F80020
:10090000000001030700008080E0E0E0E0E0E0E7B5
:10091000E3E1E0E8081C7FFCE8E8E1E161E1E1E116
:10092000E1E1E1E1E1E1E0E08080000000010101BE
:1009300001010101010101010101010100000000AB
:1009400000000000000000000000000000000000A7
:10095000000000000000FFFFFFFFFF00000000009C
:10096000FFFFFFFFFF0000000000FFFFFFFFFF0091
:100970000000E0F8F8FEFE7F1F9F87E7E1E1E1FF5E
:10098000FFFFFFFF000000FFFFE7E79F1899E1E18D
:10099000E1E1E1E1FFFFFF7F7F1F000000000000B9
:1009A0000000000000000000000000000000000047
:1009B0000000000000000000000000000000000037
:1009C0000000000000001F7F7FFFFFF8F8F8FEFE28
:1009D0007F7F1F7F7FFEFEF8F8F8FFFF7F7F1F00FD
:1009E0000000FFFFFFFFFF0606070707070707FFD7
:1009F000FFFFFFFF000000FFFFFFFF7F0607070765
:100A00000707071F7FFFFFFEF8F800000000000047
:100A100000000000000000000000000000000000D6
:100A200000000000000000000000000000000000C6
:100A3000000000000000000000010107070701019D
:100A4000000000000001010707070101000000008D
:100A500000000107071F1F00000000000000001F2A
:100A60001F07070100000007070101000000000048
:100A70000000000000010107071F00000000000047
:100A80000000000000000000000000000000000066
:100A90008040000000000000000000000000000096
:100AA0000000000000000000000000000000000046
:100AB0000000000000000000000000000000000036
:100AC0000000000000000000000000000000000026
:100AD0000000000000000000000000000000000016
:100AE0000000000000000000000000000000000006
:100AF00000000000000000000000000000000000F6
:100B000000000000000000000000000000000000E5
:100B100000000000000000000000000000000000D5
:100B200000000000000000000000000000000000C5
:100B30000000000000000000000000000000E030A5
:100B400010101010101010101010101010101010A5
:100B50001010101010101010101010101010101095
:100B60001010101030E00000000000000000000035
:100B70000000000000000000000000000000000075
:100B80000000000000000000000000000000000065
:100B90000000000000000000000000000000000055
:100BA0000000000000000000000000000000000045
:100BB0000000000000000000000000000000FF0036
:100BC000000000000000000003FFFFFFFF03000320
:100BD00003FFFF7FFEF8F8C0C0F87E7EFFFFFF0333
:100BE0000300000000FF0000000000000000000003
:100BF00000000000000000000000000000000000F5
:100C000000000000000000000000000000000000E4
:100C100000000000000000000000000000000000D4
:100C200000000000000000000000000000000000C4
:100C30000000000000000000000000000000FF00B5
:100C40000000001C7C7CFCE0E0FF7F7F1F0000E0D8
:100C5000E0FFFFE00007070F0703E0E0FFFFFFE012
:100C6000E000000000FF00000000000000000000A5
:100C70000000000000000000000000000000000074
:100C80000000000000000000000000000000000064
:100C90000000000000000000000000000000000054
:100CA0000000000000000000000000000000000044
:100CB0000000000000000000000000000000FF0035
:100CC0000000C4E464646404C4E46464E4C404E44C
:100CD000E4C404C4E4E404E46464646404C4E46454
:100CE0006464000000FF000000000000000000003D
:100CF00000000000000000000000000000000000F4
:100D000000000000000000000000000000000000E3
:100D100000000000000000000000000000000000D3
:100D200000000000000000000000000000000000C3
:100D300000000000E0F0F030F0F030F00000FF00C4
:100D40000000070F08090F000F0F0202020F000F2B
:100D50000F0103010F0F000F0909090800090B0B10
:100D60000B07000000FF0000F030F0F030F0F0E082
:100D70000000000000000000000000000000000073
:100D80000000000000000000000000000000000063
:100D90000000000000000000000000000000000053
:100DA0000000000000000000000000000000000043
:100DB00000000000070F0F07070F0F070000070CC8
:100DC00008080808080808080808080808080808A3
:100DD0000808080808080808080808080808080893
:100DE000080808080C070000070F0F07070F0F0778
:100DF00000000000000000000000000000000000F3
:100E000000000000000000000000000000000000E2
:100E100000000000000000000000000000000000D2
:100E200000000000000000000000000000000000C2
:100E300000000000000000000000000000000000B2
:100E400000000000000000000000000000000000A2
:100E50000000000000000000000000000000000092
:100E60000000000000000000000000000000000082
:100E70000000000000000000000000000000000072
:100E80000000000000000000000000000000000062
:100E90000000080B00020202000009040000010229
:100EA00002000005240010010524010101042402B0
:100EB000060524060001070581031000400904010E
:100EC00000020A0000000705020240000007058337
:100ED000024000000403090412010002EF02014075
:100EE0004123368000010102030141726475696E7D
:100EF0006F204C4C430041726475696E6F204C65E5
:100F00006F6E6172646F0000871511241FBECFEFF2
:100F1000DAE0DEBFCDBF11E0A0E0B1E0ECE7FEE437
:100F200002C005900D92AA33B107D9F728E0AAE3D1
:100F3000B1E001C01D92AD34B207E1F717E0C5E89A
:100F4000D7E004C02197FE010E943627C438D1079C
:100F5000C9F70E94B4150C943C270C9400008091B2
:100F60003A010895E9EEF3E0A0E0B8E000800EBC9D
:100F70008111012C1197A0FDFDCF0192B9F70DB49D
:100F80000895480F592F511D1416150684F5803801
:100F900091056CF597FF02C090E080E04138510563
:100FA00014F040E850E0481BFB01E770FF2721E008
:100FB00001C0220FEA95EAF777FF02C0695F7F4F11
:100FC000FB0133E0F595E7953A95E1F7F695FE2FAD
:100FD000EE27F795E795E80FF91FE751FC4F4150D1
:100FE00030F08191DF011197822B8C93F8CF089517
:100FF0004F925F926F927F928F929F92AF92BF9229
:10100000CF92DF92EF92FF920F931F93CF93DF93D4
:10101000FB01E00FF11D1E161F060CF08FC060349F
:1010200071050CF08BC0DB0177FF04C0AA27BB273A
:10103000A61BB70BA770BB27EB0177FD2796E3E054
:10104000D595C795EA95E1F777FF07C0219768E046
:1010500070E0FB01EA1BFB0BDF01E02EE694E69457
:10106000E694F12C077019F0FFEFEF1AFF0A30E059
:101070008A01AE015695542F442757954795480F3E
:10108000591F47515C4FBE01E0E8F0E05F01A81A2C
:10109000B90A88E090E03C016A1A7B0A6F3F8FEF43
:1010A00078070CF43BC090E080E04A01E0E88E0E47
:1010B000911C6F3F760709F452C0FC01E00FF11F4D
:1010C000E4916A01C80ED91EF0E02F010A2E01C07A
:1010D000440C0A94EAF7F6015080452840821097A4
:1010E000B1F06730710599F0F801E80FF91FE4914C
:1010F0006401C80ED91EF0E02F01062C02C05594E1
:1011000047940A94E2F7F601508045284082019600
:10111000821793071CF4A816B90659F66F5F7F4F24
:10112000020F131F40585F4FCB018C1B9D0B8E1578
:101130009F0524F46830710509F0B0CFDF91CF919D
:101140001F910F91FF90EF90DF90CF90BF90AF90E5
:101150009F908F907F906F905F904F900895109721
:1011600009F0C2CFD4CFFC018091E803882311F1AC
:101170003FB7F89482E08093E9002091F200822F3B
:1011800090E01816190614F481E090E0882339F0F5
:10119000289844E64093E7034091F10040832223DE
:1011A00039F02091F200211103C02BE62093E800D2
:1011B0003FBF08958FEF9FEF08952FB7F89483E016
:1011C0008093E9009091E800892F807295FF04C018
:1011D0009091F20080E4891B2FBF08958091DF0376
:1011E00081110DC082E08093DB0384E08093DC03F7
:1011F0001092DE031092DD0381E08093DF038BED1C
:1012000093E00895CF93DF931F92CDB7DEB7698344
:10121000DC01ED91FC910280F381E02D41E050E092
:10122000BE016F5F7F4F09950F90DF91CF910895B9
:1012300083E08093E9008091F200882319F08AE32B
:101240008093E80008950E94DD0890E00895CF9310
:10125000DF931F92CDB7DEB7FC018485958597FD9E
:1012600008C02FEF3FEF358724870F90DF91CF9194
:101270000895CE0101960E94B308019719F489815F
:1012800090E0F3CF8FEF9FEFF0CF0F931F93CF93AB
:10129000DF931F92CDB7DEB78C01FC018485958565
:1012A00097FF0BC0CE0101960E94B308019771F41D
:1012B000898190E0F80195878487F8018485958578
:1012C0000F90DF91CF911F910F9108958FEF9FEFB6
:1012D000F1CFFC018485958597FD0BC09FB7F894ED
:1012E00082E08093E9008091F2009FBF90E0019638
:1012F00008959FB7F89482E08093E9008091F2000E
:101300009FBF90E008954091D5035091D60320915E
:10131000D3033091D40342175307B4F49091E800FB
:101320009570E1F39091E80092FD19C08093F1006F
:101330008091D5039091D60301968F739927892BBD
:1013400019F48EEF8093E8008091D5039091D60335
:1013500001969093D6038093D50381E0089580E0B1
:101360000895DF92EF92FF920F931F93CF93DF9335
:10137000D82E8A01EB017B01E40EF51ECE15DF05A8
:1013800059F0D7FE12C0FE0184910E948309219674
:101390008111F4CF0FEF1FEFC801DF91CF911F91A3
:1013A0000F91FF90EF90DF9008958881EECF0F931B
:1013B0001F93CF93DF931F92CDB7DEB782E089836F
:1013C00042E450E062E97EE080E80E94B1090E94B8
:1013D000EE08DC0112960D911C910115110589F0A2
:1013E000D801ED91FC910280F381E02DBE016F5F89
:1013F0007F4FC801099597FD04C0F801008511854C
:10140000ECCF89810F90DF91CF911F910F910895BB
:10141000615030F02091F100FC0120830196F8CF5B
:10142000289884E68093E70308953FB7F894809165
:10143000CF039091D003A091D103B091D20326B5F0
:10144000A89B05C02F3F19F00196A11DB11D3FBFFC
:10145000BA2FA92F982F8827BC01CD01620F711DCB
:10146000811D911D42E0660F771F881F991F4A95C5
:10147000D1F708958F929F92AF92BF92CF92DF9251
:10148000EF92FF926B017C010E94150A4B015C01F7
:10149000C114D104E104F104B9F00E94150A6819DD
:1014A00079098A099B09683E73408105910580F39B
:1014B00021E0C21AD108E108F10888EE880E83E025
:1014C000981EA11CB11CE4CFFF90EF90DF90CF904D
:1014D000BF90AF909F908F9008958F929F92AF9200
:1014E000BF92CF92DF92EF92FF920F931F93CF9311
:1014F000DF936C017B018A0180910D01882309F43F
:101500005CC08091E803882309F457C08091DA0316
:1015100080FF05C08091E00082608093E000E801D8
:10152000B12C8AEFA82E93E0892E2AE3922E2097E1
:1015300011F4BB20D9F10E94DD0881110AC0AA94E0
:10154000AA20D9F161E070E080E090E00E943A0AC0
:10155000EECF8C171D0611F00CF08C2F9FB7F8946E
:101560008092E9002091E80025FD02C09FBFDFCFF7
:10157000282F30E0C21BD30BF701815020F041919E
:101580004093F100FACFE20EF31EBB2021F09092BF
:10159000E800B12CEBCF8091E80085FDE7CF909279
:1015A000E800BB24B394209709F3F3CF5D9884E659
:1015B0008093D903101611063CF081E090E0F6010B
:1015C0009383828310E000E0C801DF91CF911F91E7
:1015D0000F91FF90EF90DF90CF90BF90AF909F90D2
:1015E0008F900895AF92BF92CF92DF92EF92FF92C9
:1015F0000F931F93CF93DF936C017B018B01040F3B
:10160000151FEB015E01AE18BF08C017D10759F0D6
:101610006991D601ED91FC910190F081E02DC60118
:101620000995892B79F7C501DF91CF911F910F9112
:10163000FF90EF90DF90CF90BF90AF9008952091F2
:101640004101E0913F01F0914001CF01029690935A
:10165000400180933F01222319F0859194910895D0
:10166000808191810895CF92DF92EF92FF92CF9384
:10167000DF930E941F0B811520E8920791F480915F
:1016800071008D7F80937100109291004698479869
:1016900010924D02DF91CF91FF90EF90DF90CF90AD
:1016A000089521E020934D02813020E8920751F403
:1016B00080913D0190913E019093400180933F01C4
:1016C0000E941F0B97FD05C020913C01222309F4C5
:1016D00054C020913B01211150C021E020934201D0
:1016E000EC01DF77209709F04BC081E08093430144
:1016F00046983FE9C32E3FE0D32EE12CF12CCAEFF0
:10170000D0E0E0914708F09148080995811103C0A5
:1017100081E08093430180914201882329F08091E8
:101720004301882309F43FC047980E941F0B00978C
:10173000F1F19C01DE010E943124DC01CB0129E0A2
:10174000B595A795979587952A95D1F71092900012
:101750002AE020939100D0929900C0929800809343
:10176000440190934501A0934601B09347018091B5
:1017700071008260809371008DCF10924201B0CFD2
:101780009E0150E040E060E472E48FE090E00E944F
:10179000DD2369017A0181E0C81AD108E108F10866
:1017A00010924301AECF4699BFCF479ABECF8FEF7D
:1017B0009FEFDC01CBCF9C01E1E7F0E090819D7FC2
:1017C000908381E0809341013093400120933F0159
:1017D00030933E0120933D010C94330B2D9A0895D4
:1017E000BC0190E080E00C943A0A8FB18095807F34
:1017F000669B88601C9B8460089510923A013E9815
:101800003F9808953E9A3F9A81E080933A01089567
:1018100090915202982329F490915302982381E0E9
:1018200009F480E00895CF93C82F0E94F50B982FFC
:101830009C2381E09C1380E0CF91089580E00C947C
:10184000B20780389105B8F460347105A0F420E146
:1018500091E061FD94E060FD990F62FD9295687FD3
:10186000269FD0011124A80FA751BC4F8C9140FF97
:1018700003C0892B8C93089590958923FBCF2F92D9
:101880003F924F925F926F927F928F929F92AF9210
:10189000BF92CF92DF92EF92FF920F931F93CF935D
:1018A000DF9300D000D0CDB7DEB77C018B01242FB1
:1018B00030E03C832B8381E090E05C01A21AB30A04
:1018C0001901319421943108220C331CB901600FA5
:1018D000711F41E0C7010E94210CB8018B819C81DE
:1018E000681B790B41E0C7010E94210C41E0B8015F
:1018F0008B819C818E0D9F1D0E94210C41E0B801BF
:10190000C7012B813C81821B930B0E94210CD12C9F
:10191000C12C81E090E09A8389832B813C81C2169F
:10192000D3060CF05DC0B7FC09C0215031093C83DF
:101930002B8332E0230E311CA20CB31C8FEFC81A8C
:10194000D80A29813A812E5F3F4F3A832983A20E1C
:10195000B31E37016C0C7D1C41E08B809C80800E97
:10196000911EB401C3010E94210C27014C185D088F
:1019700041E0B401C2010E94210C41E048018B8189
:101980009C81881A990AB401C3010E94210C41E08C
:10199000B401C2010E94210C4601800E911E41E05B
:1019A000B4016B807C806E0C7F1CC3010E94210CF3
:1019B00041E0B40127012B813C81421A530AC20144
:1019C0000E94210C48018C189D0841E0B401C3011C
:1019D0000E94210C41E0B401C2010E94210C9DCF64
:1019E0000F900F900F900F90DF91CF911F910F915B
:1019F000FF90EF90DF90CF90BF90AF909F908F902F
:101A00007F906F905F904F903F902F9008958F92AE
:101A10009F92AF92BF92CF92DF92EF92FF920F937D
:101A20001F93CF93DF936D3089F0C0905002D09018
:101A300051026A30D1F410924F0210924E0288E0A7
:101A4000C80ED11CD0925102C092500281E090E0A9
:101A5000DF91CF911F910F91FF90EF90DF90CF908A
:101A6000BF90AF909F908F90089500914E0210917B
:101A70004F02E5E06E9FE0011124C952DF4F48019B
:101A8000F12CF5E0E12CFF1629F0CE010196FE01C4
:101A9000E490EC01B12CA12C4E2D4170B6016A0DE1
:101AA0007B1DC4010E94210CE694FFEFAF1ABF0A10
:101AB00088E0A816B10481F7F394EFEF8E1A9E0A1E
:101AC000F6E0FF12DECF0A5F1F4F10934F02009324
:101AD0004E02BCCF0F931F93CF93DF938C01D0E0C6
:101AE000C0E0F801EC0FFD1F6491662341F089E42A
:101AF00098E00E94070D892B11F02196F2CFCE01BC
:101B0000DF91CF911F910F910895DF92EF92FF9295
:101B10000F931F93CF93DF937C01D22E8B01040F81
:101B2000111DEB0177FF02C0D0E0C0E0C801013415
:101B3000110514F080E490E0C817D9073CF44D2D4E
:101B4000BE01C7010E94210C2196F0CFDF91CF91F9
:101B50001F910F91FF90EF90DF900895EF92FF9209
:101B60000F931F93CF93DF937C018B01C42FD22F50
:101B70000E94C107B8016D0F711D615071094C2F92
:101B8000C7010E94C10721E04D2FB801C7010E9483
:101B9000850DC7018C0F911D21E04D2FB8010197D4
:101BA000DF91CF911F910F91FF90EF900C94850DD5
:101BB000CF92DF92EF92FF920F931F93CF93DF9319
:101BC0006B01122FEC017C01E40EF11CCE15DF0538
:101BD00044F4202F412FB601CE010E94850D21969D
:101BE000F5CFDF91CF911F910F91FF90EF90DF9094
:101BF000CF9008953F924F925F926F927F928F9213
:101C00009F92AF92BF92CF92DF92EF92FF920F938B
:101C10001F93CF93DF934B01322E6C0127E0C20E4E
:101C2000D11C2C0123E0420E511CEA017C01E41A74
:101C3000F50A3B0187E0680E711C5701AC0EBD1E12
:101C4000311001C0560110E000E0888190E0002EC4
:101C500002C0959587950A94E2F780FF0EC041E097
:101C6000B401600F711FC5010E94210C41E0B30156
:101C7000601B710BC5010E94210C0F5F1F4F0830C4
:101C8000110519F721E0C21AD1082196C414D50410
:101C9000A1F6DF91CF911F910F91FF90EF90DF9010
:101CA000CF90BF90AF909F908F907F906F905F90FC
:101CB0004F903F900895089590E080E008958F92AE
:101CC0009F92AF92BF920F931F93CF93DF93CDB7A5
:101CD000DEB7A1970FB6F894DEBF0FBECDBF19A235
:101CE000423008F44AE08E010F5D1F4F842E912C84
:101CF000B12CA12CA50194010E940F24E62FB9015B
:101D0000CA01EA3044F5E05DD801EE938D01232B42
:101D1000242B252B79F790E080E0109769F0FD01E6
:101D200001900020E9F73197AF014A1B5B0BBD0121
:101D300089E498E00E94F20AA1960FB6F894DEBFFB
:101D40000FBECDBFDF91CF911F910F91BF90AF908C
:101D50009F908F900895E95CD7CFCF92DF92EF925A
:101D6000FF92CF93DF936C01990FEE08FF08F7FE07
:101D700019C06DE289E498E00E94070DEC01662726
:101D80007727CB016C197D098E099F094AE00E94D3
:101D90005F0E8C0F9D1FDF91CF91FF90EF90DF9032
:101DA000CF9008954AE0C701B601DF91CF91FF902F
:101DB000EF90DF90CF900C945F0E0C94C723CF92DE
:101DC000DF92EF92FF926B017C01C114D104E10418
:101DD000F10441F00E946F23A70196010E94DD23C8
:101DE0006B017C01C701B601FF90EF90DF90CF90AF
:101DF00008954F925F926F927F928F929F92AF92CF
:101E0000BF92CF92DF92EF92FF920F931F93CF93E7
:101E1000DF936091890370918A0380918B03909185
:101E20008C030E9424256B016091850370918603C9
:101E300080918703909188030E942425CB0121E0A3
:101E400049E953E0B6010E94FA0D80914C028823C3
:101E500009F47CC180913002882309F477C1609134
:101E600028027091290280912A0290912B020E94EF
:101E700024252B01EB0160912402709125028091B1
:101E80002602909127020E9424256B018091230253
:101E9000882309F41CC190904B018CE390E08919D0
:101EA000910963E070E00E942227EB011C161D06D9
:101EB000ACF4520188E0A80EB11C8601085F1F4FE8
:101EC000462FB501C8010E943F0CC630D10534F041
:101ED0004C2F4450B501C8010E943F0C90FC2CC00F
:101EE00064E170E080E090E00E94DF0E4B0164E16D
:101EF00070E080E090E00E94DF0E840C951CC6012B
:101F0000860F971F41E0B4010E94210C64E170E04C
:101F100080E090E00E94DF0E4B0164E170E080E021
:101F200090E00E94DF0E480C591CC601860F971FD7
:101F300041E0B2010E94210CC9E7D1E096EAE92E06
:101F400091E0F92E88858823A1F06C817D818E81B6
:101F50009F810E9424254B01688179818A819B8120
:101F60000E942425CB0101E022E044E0B4010E945C
:101F7000D80D2996EC16FD0629F7CCE4D1E089E7C7
:101F8000E82E81E0F82E88858823A1F06C817D8180
:101F90008E819F810E9424254B01688179818A81ED
:101FA0009B810E942425CB0101E022E042E0B401A4
:101FB0000E94D80D2996EC16FD0629F780914B0258
:101FC000882359F120E030E040E050E4609147027E
:101FD000709148028091490290914A020E944024E7
:101FE0000E9424256B01609143027091440280910C
:101FF0004502909146020E94242570934F026093FF
:102000004E02D0925102C092500241E050E067E38C
:1020100071E089E498E00E94F20A00E029E040E8DB
:1020200070E060E090E080E00E94D80D10924F02D6
:1020300010924E02109251021092500284ED90E0E4
:102040000E946A0D80919203909193030E94AD0EBD
:1020500088E290E090934F0280934E0210925102DA
:102060001092500280914C02882309F4A4C08DEC98
:1020700090E00E946A0D84E690E090934F02809376
:102080004E021092510210925002609154027091CF
:10209000550280915602909157024AE00E945F0ECD
:1020A00041E069E070E090E080E0DF91CF911F9126
:1020B0000F91FF90EF90DF90CF90BF90AF909F90E7
:1020C0008F907F906F905F904F900C94C10744E287
:1020D000A42E42E0B42EEEE0CE0ED11C3201FEE082
:1020E0006F0E711CF12CE12CF501848990E00E2C0F
:1020F00002C0959587950A94E2F780FF14C04701C6
:10210000880C991CB4016C0F7D1F01E022E042E0B5
:10211000C6010E94D80DB3016819790922E042E096
:10212000C6010E94D80DFFEFEF1AFF0A88E0E816FB
:10213000F104D1F6EFEFAE1ABE0AF2E0CF1AD108E1
:1021400088E2A81682E0B80669F6F6CEC6EAD1E0C3
:1021500002E212E02AE0E22EF12C8C858823F1F0D5
:102160006C817D818E819F810E9424252B01688155
:1021700079818A819B810E942425CB012D8D222388
:1021800091F02E8DA701421B51091416150634F447
:10219000B2016C5F7F4F04960E943F0C6F960C1744
:1021A0001D07D9F6C9CE20E0AE014C5E5F4FB201EB
:1021B0000E94FA0DF3CF8AEC90E00E946A0D6091C4
:1021C000010170E090E080E04AE00E945F0E53CF92
:1021D0008F929F92AF92BF92CF92DF92EF92FF9237
:1021E000CF93DF93C9E5D2E0C12CD12CE12C83E45D
:1021F000F82E288539854A855B85688179818A81B1
:102200009B810E9440244B015C0120E030E0A90149
:102210000E94AD2487FD26C088829982AA82BB8253
:102220006C817D818E819F810E9424254B01688174
:1022300079818A819B810E942425CB0141E0B401F0
:102240000E94210C2C9683E0C538D80791F6DF91C7
:10225000CF91FF90EF90DF90CF90BF90AF909F9085
:102260008F900895C882D982EA82FB8260E470E090
:1022700080E090E00E94DF0E0E945C256C837D83ED
:102280008E839F8363E070E080E090E00E94DF0E29
:102290006F5F7F4F8F4F9F4F0E945C2520E030E0A3
:1022A00040E251E40E94B224688779878A879B873D
:1022B000B7CFCF92DF92EF92FF920F931F93CF93FE
:1022C000DF9362E070E080E090E00E94DF0E6E5FDE
:1022D0007F4F8F4F9F4F6093A903C5EAD3E08E01D4
:1022E00068E770E080E090E00E94DF0EF801619303
:1022F0008F01F3E0093A1F0799F762E070E080E090
:1023000090E00E94DF0E6C5F7F4F8F4F9F4F609376
:10231000B2030EEA13E060E071E080E090E00E941A
:10232000DF0EF80161938F01F3E0023B1F0799F77D
:1023300063E070E080E090E00E94DF0E6A5F7F4F14
:102340008F4F9F4F6093BB0307EB13E064EC70E08B
:1023500080E090E00E94DF0E645C7F4F8F4F9F4FC4
:10236000F80161938F01F3E00B3B1F0779F700EC55
:1023700013E06C8170E090E080E00E945C2520E03A
:1023800030E040E85EE30E9411269B01AC0163E36C
:1023900073E383E390E40E9440246B017C012DEC05
:1023A0003CEC4CE45FE30E94AD2487FD11C0CD827C
:1023B000DE82EF82F88629960C171D07D1F6DF9191
:1023C000CF911F910F91FF90EF90DF90CF900895E4
:1023D0008DEC9CECACE4BFE38D839E83AF83B88728
:1023E000EACF0F931F93CF93DF93EC018C010C5F27
:1023F0001F4F60E071E080E090E00E94DF0E699383
:10240000C017D107B1F7DF91CF911F910F910895B8
:102410001F920F920FB60F9211248F939F9380916A
:10242000E1009091E100937F9093E10083FF0FC062
:102430001092E90091E09093EB001092EC0092E38F
:102440009093ED001092E80398E09093F00082FFE3
:1024500022C093E09093E9009091F200992319F043
:102460009AE39093E8009091D903992341F09091D9
:10247000D90391509093D903911101C05D9A909125
:10248000E703992341F09091E70391509093E7037C
:10249000911101C0289A84FF18C08091E2008E7EBD
:1024A00081608093E2008091E1008F7E8093E10063
:1024B0008091DA038E7E80618093DA039F918F9101
:1024C0000F900FBE0F901F90189580FFF7CF80914F
:1024D000E2008E7E80618093E2008091E1008E7E3A
:1024E0008093E1008091DA038E7E8160E5CF1F92B8
:1024F0000F920FB60F921124CF92DF92EF92FF92BC
:102500000F931F932F933F934F935F936F937F93FB
:102510008F939F93AF93BF93EF93FF93CF93DF93EB
:10252000CDB7DEB76C97DEBFCDBF1092E9008091CA
:10253000E80083FF25C068E0CE0145960E94080AA6
:1025400082EF8093E8008D8987FF39C09091E80081
:1025500090FFFCCF982F907609F034C19E894F8967
:10256000588D2F89F88C911131C0803861F5809198
:10257000D8038093F1001092F1008EEF8093E80071
:102580006C960FB6F894DEBF0FBECDBFDF91CF9132
:10259000FF91EF91BF91AF919F918F917F916F913B
:1025A0005F914F913F912F911F910F91FF90EF906D
:1025B000DF90CF900F900FBE0F901F9018959EEF59
:1025C0009093E800C7CF1092F100D5CF913059F425
:1025D0008111D3CF4130510581F68091D8038D7F91
:1025E0008093D803CACF933049F48111C6CF4130CC
:1025F000510519F68091D8038260F2CF953041F4ED
:102600008091E80080FFFCCF20682093E300B5CFE5
:10261000963009F0A9C00B8D1C8D22E01092E900C4
:102620001092D6031092D503F2122EC01092D4034A
:102630001092D3030E94D7091F8299E09983FA82EE
:1026400091E09E8390EA98879AEF99872091D5032D
:102650003091D603275F3F4F3C832B838D831092AD
:10266000E9001092D6031092D5031093D40300937F
:10267000D30349E050E0BE016F5F7F4F80E00E94CE
:10268000B1090E94D70979CF1093D4030093D303E3
:102690000E94EE08DC0112960D911C9101151105A6
:1026A00009F451C1D801ED91FC910480F581E02D30
:1026B000BE016B5E7F4FC8010995009709F03EC1CE
:1026C000F80100851185EACFF3E0FF120EC08F8973
:1026D000882309F440C0823061F440E860E186EF6D
:1026E0009EE00E945415811148CF81E28093EB0057
:1026F00047CF813029F440E86BE08AEE9EE0F1CFCD
:10270000833099F70E94EE08DC011296ED90FC9060
:102710008E010F5F1F4F6801E114F10479F0D701BA
:10272000ED91FC910680F781E02DB801C701099574
:10273000080F111DF701E084F184EECFD8011C923F
:10274000F60101900020E9F73197BF016C197D096E
:1027500040E0C601C6CF64ED7EE0FB01449150E04D
:1027600080E80E94B10909CF973009F4BECF9830B4
:1027700021F481E08093F10000CF993009F0FDCE83
:10278000837009F0B2CFE3E1F1E081E031E096E35C
:102790002191222371F08093E9003093EB00DF0157
:1027A00011972C912093EC009093ED008F5F873070
:1027B00079F78EE78093EA001092EA008F89809380
:1027C000E803DBCE8B8D9C8D1092E9001092D6032E
:1027D0001092D5039093D4038093D303898D8111F4
:1027E00092C08E899D89913A49F4813209F07DCF5A
:1027F00047E050E066E071E080E0B3CF913209F04D
:1028000074CF833269F48F89988DB0E0A0E0809313
:10281000020190930301A0930401B0930501ADCE92
:10282000803269F48091E80082FFFCCF67E086E0A7
:1028300091E00E94080A8BEF8093E8009ECE8232DE
:1028400009F09BCE8F8980930D01EEEFFFE7859114
:1028500094918B3F9C4D51F1E0E0F8E080910601AE
:1028600090910701A0910801B0910901803B94402B
:10287000A105B105F1F480910D0180FD1AC0EE3F74
:102880008AE0F80789F587E797E79183808380914D
:1028900060008093D70388E19BE00FB6F894A89579
:1028A000809360000FBE9093600067CEEEEFFAE079
:1028B000D5CF808191818737974709F05ECEA89563
:1028C000809160008861809360008091D70380933D
:1028D0006000EE3F2AE0F20789F08091FE0A9091B5
:1028E000FF0A9183808349CE808191818737980741
:1028F00051F29093FF0A8093FE0AC5CF1092FF0A0F
:102900001092FE0A3ACE0E94EE08DC0112960D915A
:102910001C910115110509F4E8CED801ED91FC9147
:102920000190F081E02DBE016B5E7F4FC8010995DB
:10293000811123CEF80100851185EBCF18161906F9
:102940000CF41BCED2CEF1E0FF12BECE68ED7EE0DD
:1029500004CF1F920F920FB60F9211242F933F9323
:102960008F939F93AF93BF938091CB039091CC03B0
:10297000A091CD03B091CE033091CA0323E0230F81
:102980002D3758F50196A11DB11D2093CA038093E0
:10299000CB039093CC03A093CD03B093CE0380914F
:1029A000CF039091D003A091D103B091D2030196AF
:1029B000A11DB11D8093CF039093D003A093D103A9
:1029C000B093D203BF91AF919F918F913F912F917F
:1029D0000F900FBE0F901F90189526E8230F0296B8
:1029E000A11DB11DD2CF1F920F920FB60F921124CD
:1029F0002F933F934F935F936F937F938F939F9307
:102A0000AF93BF93EF93FF93809144019091450161
:102A1000A0914601B0914701892B8A2B8B2B09F499
:102A200040C08091430181110BC088B190E4892797
:102A300088B980914201882319F088B1805888B9FB
:102A40008091440190914501A0914601B0914701C8
:102A5000181619061A061B069CF4809144019091E1
:102A60004501A0914601B09147010197A109B10923
:102A70008093440190934501A0934601B093470190
:102A8000FF91EF91BF91AF919F918F917F916F9146
:102A90005F914F913F912F910F900FBE0F901F901C
:102AA00018950E94330BECCFEF92FF920F931F9378
:102AB000CF93DF93F82E192FE62E042F81E0860F97
:102AC000880F0E94830983E00E948309CF2DD12FB4
:102AD000EC0EFD2EF11CCE15DF05B9F007FF13C07B
:102AE000FE0184910E948309182F80E00E948309CF
:102AF000812321968111EFCFDF91CF911F910F910B
:102B0000FF90EF9008958881EDCF81E0F5CFE9EE59
:102B1000F7E01382128288EE93E0A0E0B0E08483B5
:102B20009583A683B7838DE191E0918380838FEFB6
:102B30009FEF95878487E9E4F8E0138212828FE2A1
:102B400091E0918380838FEA97E090934808809387
:102B5000470880E090E8909346088093450846989F
:102B60003E9A47983F9A0895CF93DF9300D000D0C4
:102B7000CDB7DEB7789484B5826084BD84B58160BA
:102B800084BD85B5826085BD85B5816085BD809138
:102B90006E00816080936E001092810080918100B0
:102BA00082608093810080918100816080938100A8
:102BB000809180008160809380008091910082608C
:102BC0008093910080919100816080939100809129
:102BD00090008160809390008091C1008460809318
:102BE000C1008091C10082608093C1008091C100CA
:102BF00081608093C1008091C30081608093C30095
:102C00008091C00082608093C0008091C20081608A
:102C10008093C20080917A00846080937A008091D2
:102C20007A00826080937A0080917A00816080933C
:102C30007A0080917A00806880937A001092E8038D
:102C40001092D8031092DA038091D70081608093AC
:102C5000D70080EA8093D80089B5806189BD89B5A5
:102C6000826089BD09B400FEFDCF61E070E080E0C4
:102C700090E00E943A0A8091D8008F7C8061809316
:102C8000D8008091E000807F8093E0008091E10097
:102C90008E7E8093E1008DE08093E200559A209A29
:102CA00081EC80937C0085B1806F85B984B1877E8B
:102CB00084B984B1876E84B95E9A5F988AB1806D59
:102CC0008AB9769A6E9881B3806F81BB899880B3F8
:102CD0008D7080BB80E58CBD81E08DBD85E090E08E
:102CE0000E94F00B5F9A85E090E00E94F00B5E98E6
:102CF0005C98E7E8F6E084E996E024912EBD0000B8
:102D00000DB407FEFDCF31968E179F07B1F75C9A81
:102D100081E8809364008091650081608093650004
:102D20000E941E0C80E80E94130C8823A9F05C9876
:102D300085EA8EBD00000DB407FEFDCF5C9A2E988B
:102D40002F982D988091640080628093640081E0C8
:102D500083BF889513BEFCCF84E00E94130C8823A8
:102D600009F448C02D9884E80E94130C8823E1F0F0
:102D70000E94EE0B88EC90E00E94F00B2F9882E00E
:102D800090E00E94C7238F3F29F06FEF82E090E030
:102D90000E94CF2384EF91E00E94F00B2F9A84E8E9
:102DA0000E94130C8111FBCF84E10E94130C882335
:102DB000E1F00E94EE0B88EC90E00E94F00B2E9860
:102DC00082E090E00E94C723882329F060E082E03F
:102DD00090E00E94CF2384EF91E00E94F00B2E9AA6
:102DE00084E10E94130C8111FBCF88EC90E00E94DB
:102DF000F00BB2CF0E94EE0B82E090E00E94DD0E5D
:102E0000882309F4E6C00E94020C81E090E00E9451
:102E1000DD0E182F147081FF10C011112E9821EFB4
:102E20003FEF3A83298380E40E94130C882309F43E
:102E3000D3C02E9A2F9A0E94EE0B82E390E00E945C
:102E4000F00B0E94F50B8111F8CF80E18093000117
:102E5000809164008E7F8093640080917A0080640A
:102E600080937A0080917A0086FDFCCF00917800F3
:102E7000109179000E94150AAB01BC01C801B0E0B5
:102E8000A0E0DC01992788278C019D01040F151F04
:102E9000261F371FC901B8012091640021602093CB
:102EA0006400611571058105910511F00E94BE2332
:102EB0008091C20381110E94020C88EC90E00E9474
:102EC000C7238093C30389EC90E00E94C7238093BB
:102ED000C4038AEC90E00E94C7238093C5038BEC67
:102EE00090E00E94C7238093C6038091C303909112
:102EF000C403A091C503B091C6038F3F9F4FAF4F4E
:102F0000BF4F41F41092C3031092C4031092C50343
:102F10001092C6030E94591159E5252E52E0352E14
:102F200060E870E080E090E00E94DF0E0E945C2587
:102F3000D1016D937D938D939C93139760E470E022
:102F400080E090E00E94DF0E0E945C25F101648326
:102F500075838683978363E070E080E090E00E9451
:102F6000DF0E6F5F7F4F8F4F9F4F0E945C2520E0E9
:102F700030E040E251E40E94B224D10118966D93F2
:102F80007D938D939C931B97BCE02B0E311CE5E841
:102F9000F3E0E215F30521F666246394712C2FB754
:102FA000F8948091CB039091CC03A091CD03B09184
:102FB000CE032FBF009148010983002309F472C09A
:102FC0001092480180E090E0892B49F30E940000B4
:102FD000E3CF0E94FD0B19CF112339F049815A81AB
:102FE0004430510511F42E9A2F9881E00E94B207C7
:102FF00000E128E547ED55E069817A8184E190E0C0
:103000000E94F8070E941E0C8FE090E00E94F00BD7
:1030100089819A8101969A838983499709F003CF20
:10302000112311F02F9A2D9880E991E00E94F00B66
:103030000E94EE0B81E090E00E94DD0E80FFFDCE4D
:103040008AE090E00E94DD0E9FEF980F9E3F08F00F
:10305000F4CE22E330E030934F0220934E0228E377
:1030600030E030935102209350020BE010E01A83BD
:103070000983682F89E498E00E94070D89819A816D
:103080000E94DD0E09811A810F5F1F4F1A83098389
:103090000131110571F70E941E0C88EE93E00E9429
:1030A000F00BCBCE20914901182F121B212F30910C
:1030B0000001131748F42F5F231708F083CF81E036
:1030C00083BF889513BE7ECF21E020934801809373
:1030D00049018091C0039091C10301969093C1036F
:1030E0008093C00380915302809352020E94F50B9B
:1030F00080935302E9EEF3E0298121112FEF0024A0
:1031000021932193219321930394D1F7109251029B
:103110001092500210924F0210924E028091C803FA
:103120009091C9038230910509F48DC148F400974C
:1031300009F4BCC0019709F4D9C00E941E0C42CF0B
:103140008430910511F40C949C2208F402C3059775
:10315000A1F709E512E01A830983A981BA811496BF
:103160006D917D918D919C9117970E9424256B0103
:10317000E981FA8160817181828193810E94242595
:10318000CB0141E0B6010E94210C09811A81045F44
:103190001F4F1A83098320163106F9F685E290E065
:1031A00090934F0280934E0284E190E090935102FD
:1031B000809350028FEE96E00E946A0D28E230E084
:1031C00030934F0220934E0283E290E0909351029D
:1031D0008093500287EE96E00E946A0D609154023F
:1031E0007091550280915602909157024AE00E94D8
:1031F0005F0E8AE090E090934F0280934E0282E34C
:1032000090E0909351028093500284ED96E00E94EA
:103210006A0D8091540290915502A0915602B0918E
:1032200057024091C3035091C4036091C50370914C
:10323000C603481759076A077B0720F58093C30325
:103240009093C403A093C503B093C60303EC13E0AB
:1032500048EC50E05A834983D801FD908D01898163
:103260009A810E94C723F81629F06F2D89819A81CF
:103270000E94CF23E981FA813196FA83E983EC3CFD
:10328000F10551F788E00E94080C882309F455CF16
:103290007092C9036092C8038091C203882309F425
:1032A0004CCF8BE297E00E94DB0B47CF00E420E895
:1032B00040E95AE070E060E090E080E00E94F807AA
:1032C00000E02AE04AE070E060E090E080E00E94E8
:1032D000D80D8091C7038F5F8093C7038D3308F4A7
:1032E0002CCF7092C9036092C80327CF00E020E47E
:1032F00040E870E060E090E080E00E94D80D05E3D7
:1033000020E74EE757E070E060E088E090E00E9440
:10331000F80700E025E345E070E060E088E090E039
:103320000E94D80D0E94E81028E040E868E370E0B1
:1033300090E080E00E94D80D10924F0210924E0251
:1033400049E350E050935102409350028AE797E0DE
:103350000E946A0D6091C3037091C4038091C503FC
:103360009091C6034AE00E945F0E82E590E0909340
:103370004F0280934E0289E390E090935102809334
:10338000500285E797E00E946A0D1091C2031983ED
:1033900082E797E0111102C08EE697E00E946A0D65
:1033A0008091C0039091C1036CE370E00E940E27EE
:1033B0004E97C8F400E029E04AE56EE270E084E14F
:1033C00090E00E94D80D86E190E090934F028093A8
:1033D0004E028FE290E090935102809350028DE56F
:1033E00097E00E946A0D1981112341F080914D02EE
:1033F000811104C08BE297E00E94DB0B84E00E9405
:10340000080C882371F08091C20391E08927809392
:10341000C2038823A9F00E94020C8BE297E00E946D
:10342000DB0B88E00E94080C882309F486CE0E94FA
:10343000591182E090E09093C9038093C8037DCE38
:103440000E94FD0BEECF0E94E81000E028E048E566
:1034500070E060E084E190E00E94D80D8091C203AA
:10346000882341F080914D02811104C08BE297E0E6
:103470000E94DB0B2EE130E030934F0220934E028E
:1034800010925102109250028FE197E00E946A0D53
:1034900035EAC32E33E0D32E42E150E05A8349830C
:1034A000F12CE12C00E02CE04CE066E170E0898139
:1034B0009A810E94D80D21E0A60169E170E089811E
:1034C0009A8102960E94FA0D8091A403082E000CA6
:1034D000990B8E159F0549F420E140E166E170E00B
:1034E00089819A8102970E94AE0DA980BA8053E02B
:1034F000A51AB10800E024E149E16DE270E0C501E0
:103500000E94D80DB0924F02A0924E028DE290E040
:1035100090935102809350028CE197E00E946A0DD3
:10352000D60114966C9170E090E080E04AE00E9431
:103530005F0EB0924F02A0924E02E6E3F0E0F093ED
:103540005102E093500289E197E00E946A0D20E069
:1035500030E040E251E4D60115966D917D918D9158
:103560009C9118970E9411260E942425CB010E944D
:10357000AD0EBFEFEB1AFB0AE981FA81B896FA8328
:10358000E983F9E0CF0ED11C03E0E016F10409F065
:1035900089CF80E40E94080C882359F08091A4030D
:1035A000082E000C990B0196B7010E9422278093E8
:1035B000A40380E20E94080C882361F08091A40398
:1035C000082E000C990B029663E070E00E942227FF
:1035D0008093A40388E00E94080C882309F4B3C0F8
:1035E0003091A40329E03203F0011124EB55FC4F84
:1035F000A9E9B3E001900D922A95E1F710925402E7
:103600001092550210925602109257028FE080934A
:10361000010110924C0280E090E0A0E2B1E48093BE
:10362000850390938603A0938703B093880320E0DB
:1036300030E040EF51E42093890330938A034093B4
:103640008B0350938C0380919D0390E090939303A0
:103650008093920310924B02109230021092230238
:103660008CE3809322021092B2011092C301109257
:10367000D1011092E2011092F00110920102109219
:103680000F02109220021092810110928A01109272
:10369000930110929C011092A50110925401109276
:1036A0005D011092660110926F011092780109E598
:1036B00012E01A83098360E870E080E090E00E94E5
:1036C000DF0E0E945C25A981BA816D937D938D9355
:1036D0009C93139766E370E080E090E00E94DF0E19
:1036E000665F7F4F8F4F9F4F0E945C25E981FA8173
:1036F000648375838683978363E070E080E090E065
:103700000E94DF0E6F5F7F4F8F4F9F4F0E945C259F
:1037100020E030E040E251E40E94B224A981BA8165
:1037200018966D937D938D939C931B971C96BA83EB
:10373000A9832A163B0609F0BECFE3E0F0E0F09340
:10374000C903E093C80384E00E94080C8111C9CD2D
:10375000F4CC0E94E810809123028823E9F1809143
:103760004B01882371F0815080934B010E94F90E28
:1037700084E00E94080C882309F4DFCC84E090E008
:103780005ACE8091540290915502A0915602B09168
:1037900057028C599F4FAF4FBF4F80935402909365
:1037A0005502A0935602B093570210924C02109209
:1037B00030028FE080930101109223028CE380930A
:1037C00022021092540110925D0110926601109233
:1037D0006F0110927801CACF80912202882319F0DC
:1037E00081508093220280E80E94130C882331F1DB
:1037F000C0908903D0908A03E0908B03F0908C03F3
:1038000020E030E040E251E4C701B6010E940C26FE
:103810001816A4F420919E0330919F034091A003B9
:103820005091A103C701B6010E944024609389030F
:1038300070938A0380938B0390938C0380E10E94A2
:10384000130C882331F1C0908903D0908A03E09053
:103850008B03F0908C0320E030E040E652E4C70197
:10386000B6010E94AD2487FF14C0A70196016091A4
:103870009E0370919F038091A0039091A1030E94E9
:1038800041246093890370938A0380938B03909300
:103890008C0380E20E94130C882329F1C0908503D9
:1038A000D0908603E0908703F090880320E030E01A
:1038B000A901C701B6010E940C261816A4F4209194
:1038C0009E0330919F034091A0035091A103C70133
:1038D000B6010E9440246093850370938603809311
:1038E00087039093880380E40E94130C882331F1AE
:1038F000C0908503D0908603E0908703F090880302
:1039000020E030E04CED52E4C701B6010E94AD2446
:1039100087FF14C0A701960160919E0370919F03D9
:103920008091A0039091A1030E944124609385039C
:1039300070938603809387039093880380914A0154
:10394000882319F0815080934A0188E00E94130C6B
:10395000882309F449C080914A01811145C08091B2
:10396000C203882321F08CEC96E00E94DB0BE9E790
:10397000F1E090E080E020852111D3C029E0289F6C
:103980008001299F100D112407581E4F1A830983A7
:1039900020E030E040E051E46091850370918603BF
:1039A00080918703909188030E944124D8016D93F0
:1039B0007D938D939C93139720E030E040E450E496
:1039C0006091890370918A0380918B0390918C039D
:1039D0000E944124F801648375838683978381E084
:1039E00080878CE080934A0109E711E01A830983FC
:1039F00006EA11E029E7422E21E0522ED201189664
:103A00008C9118978823D1F020E030E040E450E416
:103A10006D917D918D919C910E944124F201608372
:103A200071838283938320E030E040E053E40E947E
:103A30000C2618161CF4D20118961C92B9E04B0EF5
:103A4000511C04151505D1F680914B02882309F409
:103A500085C020E030E040E05FE360914302709178
:103A6000440280914502909146020E9440246B01DD
:103A70007C01C0924302D0924402E0924502F0924F
:103A8000460220918503309186034091870350912F
:103A900088030E9440244B015C0120E030E0A90132
:103AA0000E940C2618160CF043C020E030E040EED7
:103AB00050E4C501B4010E94AD2487FF44C02091A9
:103AC000890330918A0340918B0350918C0360915C
:103AD0004702709148028091490290914A020E94E7
:103AE00040244B015C0120E030E0A9010E940C263B
:103AF00018160CF04AC120E030E040EE50E4C50159
:103B0000B4010E94AD2487FF1EC080919203909162
:103B100093030196909393038093920310924B0228
:103B200012C0019639968530910509F024CF5CCFFB
:103B300020E030E040EE50ECC501B4010E940C26BC
:103B400018160CF4BCCF20E030E040E251ECC70185
:103B5000B6010E94AD2487FD10924B0280914C0269
:103B6000882309F4ADC18091300281114DC01092BB
:103B7000B2011092C3011092D1011092E201109291
:103B8000F0011092010210920F021092200281E0C7
:103B90008093300200E010E022E033E4009324023E
:103BA00010932502209326023093270220E030E074
:103BB00040EF51E4209328023093290240932A02D7
:103BC00050932B0220932C0230932D0240932E020F
:103BD00050932F024EE150E0509332024093310255
:103BE000109234021092350210923602109237026F
:103BF00088E392E00E94F1118091C203882321F0B2
:103C000080EC96E00E94DB0BC0902402D09025024D
:103C1000E0902602F090270220E030E042ED52E4EE
:103C2000C701B6010E940C2618160CF0BAC020E09D
:103C300030E040E05FE3C701B6010E94402460939A
:103C400024027093250280932602909327020CE4AD
:103C500011E099E7E92E91E0F92ED80118968C91A0
:103C60001897882309F422C326E636E646EE5FE37A
:103C70006D917D918D919C910E9440244B015C013E
:103C8000F80180829182A282B38220E030E0A90113
:103C90000E94AD2487FF03C0D80118961C9220E033
:103CA00030E040E850E46091850370918603809194
:103CB0008703909188030E9441249B01AC01C501B8
:103CC000B4010E9440244B015C0120E030E0A901D6
:103CD0000E940C2618160CF0DEC220E030E040E80E
:103CE00050E4C501B4010E94AD2487FFDFC220E08B
:103CF00030E040E850E46091890370918A0380913C
:103D00008B0390918C030E9441249B01AC01F8012C
:103D100064817581868197810E9440244B015C01FA
:103D200020E030E0A9010E940C2618160CF058C3C0
:103D300020E030E040E850E4C501B4010E94AD2429
:103D400087FFB4C28091920390919303019790935F
:103D5000930380939203D80118961C928091C2031A
:103D6000882321F088EB96E00E94DB0B8091920380
:103D700090919303181619060CF498C2E5E0F0E050
:103D8000F093C903E093C80391C220E030E040EE15
:103D900050ECC501B4010E940C2618160CF4B5CEE7
:103DA000D2CE2AE037ED43E25DE3609134027091B8
:103DB000350280913602909137020E94412460932F
:103DC00034027093350280933602909337020E943A
:103DD0007E2620E030E040E951E40E94112620E0F8
:103DE00030E048EC51E40E9441246B017C0120E06A
:103DF00030E040E251E40E94AD2487FD4DC0C09206
:103E00002802D0922902E0922A02F0922B026EE15F
:103E100070E080E090E00E94DF0E61307105810566
:103E2000910509F014CFECE4F1E090E080E020850A
:103E300021113FC029E0289FD001299FB00D1124F6
:103E4000A45BBE4FBC83AB8380912402909125027A
:103E5000A0912602B0912702EB81FC81808391839F
:103E6000A283B38320E030E040E051E46091280277
:103E70007091290280912A0290912B020E94412484
:103E8000AB81BC8114966D937D938D939C93179712
:103E900081E018968C93DBCE80E090E0A0E2B1E464
:103EA0008093280290932902A0932A02B0932B02B8
:103EB000AECF019639968530910509F0B8CFC7CEBF
:103EC00006EA11E01C830B8311E009E0AB81BC81A1
:103ED0001C968C911C97882309F496C15D968C9151
:103EE0005D97882309F462C05E968C915E97882363
:103EF00069F081505E968C932B813C81215E3F4F0F
:103F00003C832B832252324009F7A1CEEB81FC8106
:103F10001486158E8091540290915502A0915602FC
:103F2000B09157020A96A11DB11D8093540290933F
:103F30005502A0935602B093570280910101882345
:103F400019F081508093010180910101811102C01B
:103F500010934C0280914B028111CECF6AE070E049
:103F600080E090E00E94DF0E6130710581059105CF
:103F700019F610934B02EB81FC8180819181A28123
:103F8000B3818093430290934402A0934502B0937F
:103F9000460284819581A681B781809347029093E0
:103FA0004802A0934902B0934A02A6CF20E030E035
:103FB00040E85FE3AB81BC816D917D918D919C91D7
:103FC0000E944024EB81FC81608371838283938310
:103FD0008785813061F52DEC3CEC4CE45DE3608934
:103FE0007189828993890E944124AB81BC8150965A
:103FF0006D937D938D939C9353970E947E2620E032
:1040000030E040E751E40E9411269B01AC01EB81B6
:10401000FC8160857185828593850E944124AB81F6
:10402000BC8114966D937D938D939C93179720E09C
:1040300030E040E251E4EB81FC816481758186814E
:1040400097810E94AD2487FF0AC080E090E0A0E243
:10405000B1E4EB81FC8184839583A683B78360E51B
:1040600070E080E090E00E94DF0E61307105810514
:10407000910579F5ECE4F1E090E080E020852111F4
:1040800093C0089F9001099F300D1124A901445B42
:104090005E4F7A01EB81FC8180819181A281B381A5
:1040A000FA0180839183A283B38320E030E040E86B
:1040B00050E4AB81BC8114966D917D918D919C9162
:1040C00017970E944124F701648375838683978341
:1040D0001087AB81BC812D913D914D915C91609198
:1040E00085037091860380918703909188030E94D5
:1040F00040244B015C0120E030E0A9010E940C2625
:1041000018160CF058C020E030E040EE50E4C50135
:10411000B4010E94AD2487FF59C0EB81FC8124814A
:104120003581468157816091890370918A0380911E
:104130008B0390918C030E9440244B015C0120E092
:1041400030E0A9010E940C2618160CF051C020E0A6
:1041500030E040EE50E4C501B4010E94AD2487FF79
:1041600035C08091920390919303019790939303AC
:1041700080939203AB81BC811C961C928091C203F8
:10418000882321F088EB96E00E94DB0B809192035C
:104190009091930318161906CCF0E5E0F0E0F09347
:1041A000C903E093C80312C0019639968530910582
:1041B00009F064CF8ECF20E030E040EE50ECC50136
:1041C000B4010E940C2618160CF4A7CF20E030E0B2
:1041D00040E251ECAB81BC816D917D918D919C91C0
:1041E0000E94AD2487FF88CEEB81FC81148684CEAB
:1041F00020E030E040EE50ECC501B4010E940C26F6
:1042000018160CF4AECFE2CF80912202811174CE49
:1042100068E270E080E090E00E94DF0E613071059E
:104220008105910509F068CEAB81BC811C961C9379
:104230001C975D961C925D9720E030E042E053E4CD
:104240002D933D934D935C93139763E270E080E070
:1042500090E00E94DF0E615F7F4F8F4F9F4F0E9463
:104260005C25EB81FC8160877187828793876483FB
:1042700075838683978362E070E080E090E00E941F
:10428000DF0EEB81FC81678776866586CF014496D9
:104290000E94F11131CE20E030E040E850ECC50141
:1042A000B4010E940C2618160CF421CD075F1F4F95
:1042B000E016F10609F0D1CC11E00AE0A981BA813B
:1042C00018968C91882309F480C080914C02882331
:1042D00009F492C080913002882309F48DC0C09007
:1042E0002402D0902502E0902602F090270220E0E0
:1042F00030E042ED52E4C701B6010E94AD24181629
:104300000CF463C0E981FA8180809180A280B3803F
:10431000A5019401C701B6010E94AD2487FF55C0D5
:1043200020E030E040E851E4C701B6010E9441249A
:104330009B01AC01C501B4010E94AD2487FF45C0BB
:10434000A981BA811496CD90DD90ED90FC901797DD
:104350008090280290902902A0902A02B0902B020F
:10436000A5019401C701B6010E940C2618166CF530
:1043700020E030E040E851E4C501B4010E9441244E
:104380009B01AC01C701B6010E94AD2487FF1DC08F
:104390008091310290913202019790933202809382
:1043A0003102E981FA8110861816190674F0F1E0DD
:1043B000F09323022CE320934B018091C2038823C6
:1043C00021F080EA96E00E94DB0B49815A81475F29
:1043D0005F4F5A8349834416550609F06FCFC6C90B
:1043E00020E030E040E850ECC501B4010E940C260A
:1043F00018160CF4A7CC5ACF86EAE82E81E0F82EE6
:10440000D7011C968C911C97882309F480C05D9677
:104410008C915D9781117BC020E030E040E850E452
:104420006D917D918D919C910E9441249B01AC01E5
:10443000E981FA8160817181828193810E944024A7
:104440004B015C0120E030E0A9010E940C26181607
:104450000CF052C020E030E040EA50E4C501B40165
:104460000E94AD2487FF53C020E030E040E850E4D4
:10447000D70114966D917D918D919C9117970E9413
:1044800041249B01AC01E981FA81648175818681B7
:1044900097810E9440244B015C0120E030E0A9019B
:1044A0000E940C261816ECF520E030E040EA50E4BB
:1044B000C501B4010E94AD2487FF29C0D7011D9614
:1044C0008D919C911E9701971E969C938E931D979C
:1044D000E981FA81108618161906CCF05D961C93B6
:1044E0005D975E960C938091C203882381F084E9E6
:1044F00096E00E94DB0B0BC020E030E040EA50EC7D
:10450000C501B4010E940C2618160CF4ADCFFFE1D2
:10451000EF0EF11C22E2E21622E0F20609F070CF63
:1045200054CF20E030E040EA50ECC501B4010E94D5
:104530000C2618161CF2EBCF09E512E01A8309834A
:10454000A981BA8114966D917D918D919C91179757
:104550000E9424256B01E981FA8160817181828149
:1045600093810E942425CB0141E0B6010E94210CD9
:1045700009811A81045F1F4F1A83098320163106AF
:10458000F9F60E94F90E00E023E24CE36FE070E0E0
:1045900082E290E00E94D80D23E24CE36FE070E0ED
:1045A00082E290E00E94AE0D28E230E030934F02AC
:1045B00020934E0284E190E0909351028093500248
:1045C00000915802098380E197E0002311F087E011
:1045D00097E00E946A0D28E230E030934F0220936A
:1045E0004E0240E250E05093510240935002098144
:1045F00080E097E0013011F089EF96E00E946A0DAB
:1046000080E80E94080C811105C080E10E94080C1E
:10461000882329F081E01981811B8093580288E06A
:104620000E94080C882311F40C949D188091580264
:1046300081110C94481923E030E03093C903209392
:10464000C8030C949D188F929F92AF92BF92CF9205
:10465000DF92EF92FF92CF93DF93EC016881798133
:104660008A819B81611571058105910521F464E2C0
:1046700079ED8BE597E02DE133EF41E050E00E94CA
:10468000DD2349015A019B01AC01A7EAB1E40E9474
:10469000FC236B017C01ACEEB4EFA50194010E94F8
:1046A0000A24C60ED71EE81EF91EF7FE06C081E0DA
:1046B000C81AD108E10880E8F80AC882D982EA82DB
:1046C000FB82C701B6019F77DF91CF91FF90EF90FA
:1046D000DF90CF90BF90AF909F908F9008958F9272
:1046E0009F92AF92BF92CF92DF92EF92FF92609132
:1046F0000E0170910F0180911001909111016115CF
:1047000071058105910521F464E279ED8BE597E06F
:104710002DE133EF41E050E00E94DD2349015A01D1
:104720009B01AC01A7EAB1E40E94FC236B017C0170
:10473000ACEEB4EFA50194010E940A24C60ED71E68
:10474000E81EF91EF7FE06C081E0C81AD108E1088C
:1047500080E8F80AC0920E01D0920F01E092100199
:10476000F0921101C701B6019F77FF90EF90DF90A3
:10477000CF90BF90AF909F908F90089560930E015F
:1047800070930F0180931001909311010895F9998E
:10479000FECF92BD81BDF89A992780B50895262F46
:1047A000F999FECF1FBA92BD81BD20BD0FB6F89416
:1047B000FA9AF99A0FBE01960895052E97FB1EF4FA
:1047C00000940E94F42357FD07D00E940F2407FC99
:1047D00003D04EF40C94F4235095409530952195D8
:1047E0003F4F4F4F5F4F089590958095709561951D
:1047F0007F4F8F4F9F4F08950E943124A59F900DAA
:10480000B49F900DA49F800D911D11240895B7FFB2
:104810000C94FC230E94FC23821B930B0895A1E2BD
:104820001A2EAA1BBB1BFD010DC0AA1FBB1FEE1F2A
:10483000FF1FA217B307E407F50720F0A21BB30B75
:10484000E40BF50B661F771F881F991F1A9469F7F1
:1048500060957095809590959B01AC01BD01CF014D
:104860000895A29FB001B39FC001A39F700D811D49
:104870001124911DB29F700D811D1124911D089569
:104880005058BB27AA270E9458240C94D2250E9476
:10489000C42538F00E94CB2520F039F49F3F19F44D
:1048A00026F40C94C1250EF4E095E7FB0C94BB258F
:1048B000E92F0E94E32558F3BA17620773078407AC
:1048C000950720F079F4A6F50C9405260EF4E095F2
:1048D0000B2EBA2FA02D0B01B90190010C01CA01BA
:1048E000A0011124FF27591B99F0593F50F4503E65
:1048F00068F11A16F040A22F232F342F4427585F57
:10490000F3CF469537952795A795F0405395C9F76E
:104910007EF41F16BA0B620B730B840BBAF0915026
:10492000A1F0FF0FBB1F661F771F881FC2F70EC0C5
:10493000BA0F621F731F841F48F487957795679598
:10494000B795F7959E3F08F0B0CF9395880F08F084
:104950009927EE0F9795879508950E94972508F45B
:1049600081E008950E94C6240C94D2250E94CB2594
:1049700058F00E94C42540F029F45F3F29F00C94C0
:10498000BB2551110C9406260C94C1250E94E325E9
:1049900068F39923B1F3552391F3951B550BBB276E
:1049A000AA2762177307840738F09F5F5F4F220FB3
:1049B000331F441FAA1FA9F335D00E2E3AF0E0E8AA
:1049C00032D091505040E695001CCAF72BD0FE2FF4
:1049D00029D0660F771F881FBB1F26173707480788
:1049E000AB07B0E809F0BB0B802DBF01FF27935840
:1049F0005F4F3AF09E3F510578F00C94BB250C9424
:104A000006265F3FE4F3983ED4F386957795679545
:104A1000B795F7959F5FC9F7880F911D9695879574
:104A200097F90895E1E0660F771F881FBB1F621793
:104A300073078407BA0720F0621B730B840BBA0B51
:104A4000EE1F88F7E09508950E942B256894B11118
:104A50000C94062608950E94EB2588F09F5798F045
:104A6000B92F9927B751B0F0E1F0660F771F881F73
:104A7000991F1AF0BA95C9F714C0B13091F00E948D
:104A80000526B1E008950C940526672F782F882716
:104A9000B85F39F0B93FCCF3869577956795B395B4
:104AA000D9F73EF490958095709561957F4F8F4F23
:104AB0009F4F0895E89409C097FB3EF49095809528
:104AC000709561957F4F8F4F9F4F9923A9F0F92FD4
:104AD00096E9BB279395F695879577956795B79552
:104AE000F111F8CFFAF4BB0F11F460FF1BC06F5F38
:104AF0007F4F8F4F9F4F16C0882311F096E911C04A
:104B0000772321F09EE8872F762F05C0662371F06A
:104B100096E8862F70E060E02AF09A95660F771F7E
:104B2000881FDAF7880F9695879597F90895990F5A
:104B30000008550FAA0BE0E8FEEF16161706E80767
:104B4000F907C0F012161306E407F50798F0621B88
:104B5000730B840B950B39F40A2661F0232B242B5D
:104B6000252B21F408950A2609F4A140A6958FEF7C
:104B7000811D811D089597F99F6780E870E060E0CE
:104B800008959FEF80EC089500240A9416161706E6
:104B900018060906089500240A941216130614062E
:104BA00005060895092E0394000C11F4882352F091
:104BB000BB0F40F4BF2B11F460FF04C06F5F7F4F49
:104BC0008F4F9F4F089557FD9058440F551F59F030
:104BD0005F3F71F04795880F97FB991F61F09F3FEA
:104BE00079F087950895121613061406551FF2CF13
:104BF0004695F1DF08C0161617061806991FF1CF63
:104C000086957105610508940895E894BB27662789
:104C10007727CB0197F908950E94972508F48FEF25
:104C200008950E9424260C94D2250E94C42538F0B1
:104C30000E94CB2520F0952311F00C94BB250C94F9
:104C4000C12511240C9406260E94E32570F3959F3C
:104C5000C1F3950F50E0551F629FF001729FBB2773
:104C6000F00DB11D639FAA27F00DB11DAA1F649F0F
:104C70006627B00DA11D661F829F2227B00DA11DC2
:104C8000621F739FB00DA11D621F839FA00D611D48
:104C9000221F749F3327A00D611D231F849F600D69
:104CA000211D822F762F6A2F11249F5750409AF092
:104CB000F1F088234AF0EE0FFF1FBB1F661F771F1E
:104CC000881F91505040A9F79E3F510580F00C94E9
:104CD000BB250C9406265F3FE4F3983ED4F38695FB
:104CE00077956795B795F795E7959F5FC1F7FE2B89
:104CF000880F911D9695879597F908959F930E9427
:104D000088260F9007FCEE5F0C94B1260C94C12509
:104D10000E94EB25D8F3E894E0E0BB279F57F0F022
:104D20002AED3FE049EC06C0EE0FBB0F661F771F70
:104D3000881F28F0B23A62077307840728F0B25A36
:104D4000620B730B840BE3959A9572F7803830F4FD
:104D50009A95BB0F661F771F881FD2F790480C9457
:104D6000C726EF93E0FF07C0A2EA2AED3FE049EC37
:104D70005FEB0E9458240E94D2250F90039401FCFF
:104D80009058ECEAF0E00C94D3269F3F31F091501C
:104D900020F4879577956795B795880F911D96951F
:104DA000879597F908959F938F937F936F93FF93C0
:104DB000EF939B01AC010E941126EF91FF910E949D
:104DC000E7262F913F914F915F910C941126DF932D
:104DD000CF931F930F93FF92EF92DF927B018C0191
:104DE000689406C0DA2EEF010E942426FE01E894A2
:104DF000A5912591359145915591A6F3EF010E941A
:104E00005824FE019701A801DA9469F7DF90EF902A
:104E1000FF900F911F91CF91DF910895AA1BBB1BAB
:104E200051E107C0AA1FBB1FA617B70710F0A61BAA
:104E3000B70B881F991F5A95A9F780959095BC01CB
:104E4000CD01089597FB072E16F4009407D077FD47
:104E500009D00E940E2707FC05D03EF4909581955D
:104E60009F4F0895709561957F4F0895EE0FFF1F36
:0C4E70000590F491E02D0994F894FFCF18
:104E7C00100FFFFFFFFF00E1000000000000010029
:104E8C00000000C180810000000000000002096DDC
:104E9C000A230918096909270945090000000007B8
:0A4EAC000DF20A5C0E5B0E2B0000F5
:00000001FF
